:020000040000FA
:040000006F303A28FB
:040004000034003490
:08000800A000030EA100831209
:100010008B1C32288B1032181428B21C3228643002
:10002000010203183128182800001628172818285C
:1000300019281A281B281C281D281E281F283210A2
:10004000B214A810031005190314AA0DA90DA80DC8
:10005000B10B322832152A08AF002908AE00280853
:10006000AD00B21081010B11210E8300A00E200EF5
:02007000090085
:0C007400203084008001840A80300402E7
:10008000031C3C281230B100722183160C30850508
:1000900087018312850187010730990000309A009B
:1000A000103083168E008312603083168F00831207
:1000B00000308316910000008312C830831681003F
:1000C000831231309000003083168C008312103080
:1000D0008B00B42181018E018F010B118B100B104D
:1000E0008C018B178220321998205421B40B802860
:1000F000031085190314BA0DF0303A020319F620E3
:10010000B52172286400321808000B1D08000B117D
:10011000B21032141230B100051D93283314831627
:10012000011383120800331083160117831208008D
:1001300032110130B7008B132030370783169B0034
:100140001C141A088312A400A500C030A5061030A4
:10015000370783169B001C141A088312A300003073
:10016000370783169B001C141A088312A2008B17F2
:10017000331CC02822090339A200A309A409A50938
:1001800022082D02031DF02823082E02031DF0284B
:1001900024082F02031DF02801303702031DD52843
:1001A0003E18D5283E143F148D2102303702031D1E
:1001B000DE28BE18DE28BE143F1496210330370215
:1001C000031DE7283E19E7283E153F149F21043000
:1001D0003702031DF028BE19F028BE153F14A821D0
:1001E000B70A05303702031808009B280130B60013
:1001F000B400B500B70085018701B213B021822099
:10020000B40B1529031085190314BA0DF0303A0206
:1002100003193C295030B400B51F8501B51F870173
:10022000B50B15299630B5004821321DFF28321133
:10023000331C1F292D090339AD00AE09AF092F1C4E
:10024000B2132F1CFF28B21BFF282E18FF28B2174D
:100250008B1320303707BC002F08BB005D21103006
:100260003707BC002E08BB005D2100303707BC00FB
:100270002D08BB005D218B1785018701B70AB601E8
:100280000130B50005303702031CFF28B4210800F7
:100290003708B6080319B6000319080011308500A5
:1002A00013308700B60308003F1C08003F101030D1
:1002B000BC003E08BB005D2108008B133B08831681
:1002C0001C159A0083123C0883169B0055309D0034
:1002D000AA309D009C1464009C186B291C11831289
:1002E0008B170800831610309B001C141A08831209
:1002F000BE00831620309B001C141A088312C20013
:100300000130C21BC200C2080319C2000130D5006F
:10031000D200EE30D000D10008000130D500D2006C
:10032000EE30D000D1000130BE0008000130D50011
:10033000D200EE30D000D1000230BE000800013003
:10034000D500D200EE30D000D1000430BE0008004D
:100350000130D500D200EE30D000D100BE0108003F
:100360000800B801B901080008008F080319080047
:100370008F01C10B08004208C100D50B08005608C8
:10038000D50007303E050319EC29D21BD00AD21F35
:10039000D0030A305002031CE729D0010930D21FD4
:1003A000D0005203D2007F39031DE729D10A103053
:1003B0005102031CDC29D1015022D2006022D4005A
:1003C0007022D600D500D0010930D21FD000002302
:0E03D0008500242387000800850187010800AE
:1004A00002308A0051083E1C572A883E8200BE1C3A
:1004B0005B2A883E82003E1D5F2A983E82000034FF
:1004C00002308A0051083E1C672AA83E8200BE1CEA
:1004D0006B2AB83E82003E1D6F2AB83E820000346F
:1004E00002308A0051083E1C772AC83E8200BE1C9A
:1004F0007B2AD83E82003E1D7F2AE83E82000134DE
:100510000734873407348734033483340334833413
:100520000B3403340F3407340B34033403340734EF
:10053000053487340734253483340334073489344D
:100540000B3403348F3405348B34113403340334C7
:1005500001340134023402340434043408340834DD
:10056000103410342034203440344034803480340B
:10057000083404340234803440348034103402347B
:10058000043410342034013404344034843480344E
:10059000093409340A340A34083408340834083475
:1005A0000834183408341834083418341034083433
:1005B000093429340A341A34283408340834083405
:1005C0000A34383408341A3408345834103448346F
:1005D000293409340A340A342834083408344834B5
:1005E0002834183488341834283418341034083433
:1006000003308A005008541C072B4B3E8200D41C38
:100610000B2B563E8200541D0F2B613E8200D41DD1
:10062000132B6C3E8200541E172B773E8200D41E83
:100630001B2B823E8200541F1F2B8D3E8200D41F35
:10064000232B983E8200003403308A005008541C4B
:100650002B2BA33E8200D41C2F2BAE3E8200541DB8
:10066000332BB93E8200D41D372BC43E8200541E6A
:100670003B2BCF3E8200D41E3F2BDA3E8200541F1C
:10068000432BE53E8200D41F472BF03E820000340E
:0A0696001034203401340234003423
:0A06A000003400340034003400344C
:0406AC0010343034A2
:1006B0003134333433343334333433343334333404
:0E06C2000034003400340034003400340234BC
:0606D0000334233433342F
:0806D800103420340134023417
:0C06E000003410342034013402340034A3
:0206EE001034C6
:1006F0002034013402340034003402340134203414
:020700001034B3
:0C070400103430343134333433343334A7
:080710003134303410340034A0
:06071A00333423340334E4
:0E072000023400340034023403342334333402
:10073000333400343334003433340034333400344D
:04074000333400341A
:0A07460000340034003400340234A3
:0A075000043401342034103408345E
:04075C000034003431
:1007600000340034023406340734273437343F343D
:0E07720008341834383439343D343F343F34C1
:060780003F343F343F341A
:08078800043401342034103464
:0C0790000A3404340134203410340A34DC
:02079E0008341D
:1007A000103420340134063406340134203410343B
:0207B00008340B
:0C07B40008341834383439343F343934F8
:0807C000383418340834003409
:0607CA003F3437342734F0
:0E07D0000734063406340734273437343F34F8
:1007E0003F3400343F3400343F3400343F3400346D
:0407F0003F3400345E
:084000000C00030007000100A1
:02400E00CC33B1
:10420000010003000300030003000200020002009B
:1042100002000000000000000000FF00FF00FF009F
:10422000000000000000000000000000000000008E
:104230000000C000C000C000C000FF00FF00FF0081
:104240000100C300F300CF00FF00C300F300CF0064
:10425000FF00C300F300CF00FF00FF00FF00FF00DE
:10426000FF00FF00FF00FF00FF00FF00FF00FF0056
:10427000FF00FF00FF00FF00FF00FF00FF00FF0046
:10428000FF00FF00FF00FF00FF00FF00FF00FF0036
:10429000FF00FF00FF00FF00FF00FF00FF00FF0026
:1042A000FF00FF00FF00FF00FF00FF00FF00FF0016
:1042B000FF00FF00FF00FF00FF00FF00FF00FF0006
:1042C000FF00FF00FF00FF00FF00FF00FF00FF00F6
:1042D000FF00FF00FF00FF00FF00FF00FF00FF00E6
:1042E000FF00FF00FF00FF00FF00FF00FF00FF00D6
:1042F000FF00FF00FF00FF00FF00FF00FF00AA001B
:00000001FF
